:020000040000fa
:080000000002040000000000f2
:020000040000fa
:100400006fd22000007f2200000188000000000061
:100410000c000700408922000100200011000700a5
:10042000000020000000e000020032000000020096
:10043000000000009e1e0200000000000040da00e4
:100440000000fe004440a900401220000000e0002f
:100450000300320000002000a00188004440a800f2
:100460000000060091018800800078000000eb0089
:1004700015003700e280400032a0b4009101ba00bc
:10048000e280400032a0b4009102ba00e280400055
:1004900032a0b4000002eb00472bde00f507b200eb
:1004a000602ce10004003a000059eb008301e900f0
:1004b000fdff3e00040037006128e100010032002a
:1004c0000082eb00040007001101ba000200e00006
:1004d000e8ff3a00000006003159ba008301e90044
:1004e0000c0032002159ba008301e90008003200f3
:1004f0000400e00003003a00e280400032a0b400b3
:10050000f5ff370011d9ba008301e900faff3a007c
:100510008100e800e180400032a0b4000000060045
:10052000000178001001e200030035001061a8000e
:10053000000028001021b70030088000410880002a
:100540000200e000010032000089be000000060049
:100550000a00fa0044002000b4bf9f00c0bf9f0003
:10056000d2bf9f00e3bf9f00f1bf9f006a8057008a
:1005700000c0da005fb89700efb897000080fa007b
:10058000000006000a00fa0080017800e20f500027
:1005900028003e0010698000e10f50000800320082
:1005a000802320000000e00005003200042320002a
:1005b0002523200046232000800178000400370016
:1005c0000422200025222000462220008322200031
:1005d000144090000004e000040035008009eb00a6
:1005e000144090000074a000104298001540900044
:1005f0000028a30003003a00154090000024a0004a
:10060000904298008001eb000700370015409000f1
:100610000008a300fdff320063c078000000fb006b
:10062000000b78008301e800828f5100f7ff3a0049
:100630000800370030002000b0bf9f00c3bf9f00fc
:10064000d1bf9f00e2bf9f006a80570000c0da0060
:100650006fb99700020078000080fa0000000600e1
:10066000889fbe0080047800206980000000e000c0
:1006700003003a00100007000000e0000a00350007
:10068000206980000900e00002003a0000047800c0
:10069000060037000004780009004000060007004b
:1006a0000000e00001003d000084eb00080078003d
:1006b0004f04be0000000600800078000000e0004b
:1006c00004003a0000002000206988000101780041
:1006d000060037000081eb0000002000808f5000f2
:1006e00002003e00216988000001eb000200780052
:1006f00000000600889fbe008a9fbe0001057800aa
:100700000100e0000400350008003c000000e000ab
:10071000200032000500370060001000e080180063
:1007200002003b0001f02c001a0037000004be005c
:100730006011b8006b0920000982cf000200390067
:100740000882cf000441b000694252000e0032001e
:1007500008003b0082817100610164008904d100be
:100760000884d3008b05e8000442e800f9ff3a0052
:10077000050037000804440089844c008b05e9001b
:100780000442e900fbff3a00000107000af0a7005d
:1007900001f0a0004f05be004f04be00000006009f
:1007a000889fbe008a9fbe008c1f78001d01070035
:1007b0002401330003866c006450e1002e003200f7
:1007c0006420e100330032006150e1002f0032006c
:1007d0006120e1003100320085855500eb07b00053
:1007e0000900200008042000050037000804440028
:1007f00089844c000a0031000603430087834b00c4
:100800000001530081815b00f8ff33000203be004a
:100810000800a0000804440089844c00f6ff390059
:10082000c639dd008301730001003200130020008f
:100830008904d1000884d3000998a3000500320080
:100840000800a7000300a0008904d1000884d30099
:100850008b05e8008904d1000884d3000001eb0077
:100860000281d200c900070001f0a1000cf0a7002e
:1008700001f0a000fc0037006420e100fe0032001f
:100880000801be000200be00f7ff37006120e10052
:10089000f90032006000b800f3ff370000002000cc
:1008a00001f82700f0ff370014002000f5003700a2
:1008b00003f0a200889fbe008a9fbe008c1f7800b4
:1008c000d8000700df0033006450e1004f00320021
:1008d0006420e1005200320003826c0007003b00fc
:1008e0000905d0000306d000820f54000c065d00fd
:1008f0000200390002003200890178000306780006
:100900008582550004003d000003fd008103fd00c9
:100910008502ea008b854200840f720002003b00d2
:1009200060001000e08018006011b8000005eb00c6
:100930007a28e1000a00390006007800c75ddd0072
:10094000f707b200878075002d00370082817100a3
:100950000a017800610560008180d1000080d30029
:100960008502e900f9ff3b00060440008784480047
:1009700002003b0060041400e0841c000988a3000e
:10098000070032008a817100828171006101640078
:100990008904d1000884d3008b05e80017003700d4
:1009a0000978a30013003a000b00e00013003400a4
:1009b0008b05e9000804440089844c000a44740053
:1009c0000978a3000d003a000b00e0000700340096
:1009d0008b05e9000804440089844c0001003a00ba
:1009e0000b0020000978a300f7ff32000001eb00a4
:1009f00002003700828171000a017800630007005d
:100a00000cf0a70001f0a000970037006420e1007f
:100a100002003a00838f6c00970033000801be008b
:100a20000200be0090003700889fbe008a9fbe0073
:100a30008c1f78007b0007008200330003866c0067
:100a40006450e100240032006420e10027003200fd
:100a50006150e100220032006120e10021003200fb
:100a60008b854200eb07b1000134b800003ab800b2
:100a70000804420089844a00013ab8000030b800f6
:100a80008880400009014a00040033000000400053
:100a900081804800020149008b05e900c909dd0099
:100aa000830170000100320013002000c814de0032
:100ab0004814dd004709de001200b200c808de005d
:100ac000088470003100070001f0a1000cf0a700bd
:100ad00001f0a000640037006120e10066003200f0
:100ae0000801be000200be00f7ff37006150e100c0
:100af000fcff3a0060003700f4ff2f006100370070
:100b0000040020005f0037000001be0078000700ed
:100b10000470a70003f0a1006509b10016003200bf
:100b20000d0035006828e10006003500f0ff2f00b9
:100b3000f1ff27000300e00013003b000100280044
:100b40000000050000004000818048008502e900a7
:100b5000fcff3a0008003700f88f420002003c001a
:100b60008000eb00000005008100d1000080d30070
:100b70008502e800fcff3a000300e00002003b00b1
:100b800060001000e08018000000060081002000d6
:100b9000618055000b003d000b00200061fe2f001e
:100ba0000100e1001d0034008281710061016400d8
:100bb0008904d1000884d3000000e800faff3a005d
:100bc00071002000610064000300700002006000fa
:100bd0000900320061044400e0844c000988a5004b
:100be000050032008b05e8006808e10002003a00c9
:100bf0008904d1000884d300f20f20000258e100dc
:100c000005003d00c75ddd00f907b2008980750071
:100c100008007800000006000bf827008b00780021
:100c2000000005000004be00310007000003be0004
:100c30000405be000200be002d000700844f7500b1
:100c4000000006000200be006450e100050036000e
:100c50006420e100020036000968a30001003a00a8
:100c60000800be000160a0004f0678004f05be00de
:100c70004f04be0000000600f0ff2f00f1ff270028
:100c8000f9ff3700889fbe008a9fbe00841f78004e
:100c9000e4ff07004f00780011003300f0ff2f0041
:100ca000838f6c0006003b00040565000a00a70066
:100cb0000800370009f0a6001000200008003700e7
:100cc000820f5400838f5c00030039001000200065
:100cd00001003e000000200009f0a7000000ea002b
:100ce0004f05be004f04be000000e00000000600fb
:100cf000c70ade00f107b200f50fb20008003200ab
:100d0000e1cf4200020032000170a0002400050083
:100d1000810f700001003200040805004400050046
:100d2000810f700002003a00140005008502e900fe
:100d30000000400081c04800fcff3b000170a000a3
:100d4000240005002800fa00889fbe008a9fbe008c
:100d50008c9fbe0003866b00620307000028a3007f
:100d600064003a000128a30067003a000008a300cd
:100d700062003a000108a30065003a001e009000de
:100d8000be08900081064000ed3fb100f48057009e
:100d9000ee019000111ab8008e099000311bb800c6
:100da0009e099000311cb800511db800f485570011
:100db00046000700fe0190003a0007008b85e8001e
:100dc0003e0007008e09900040000700ee019000f1
:100dd000340007008b85e800380007008e0990007a
:100de000400007009e0990001b18b80089044000cd
:100df0000a854800fe019000340007008b85e8005a
:100e000038000700ee019000300007008e099000c6
:100e10001b18b800890440000a8548000a98a300fe
:100e200008003a000402420085824a0006034b0093
:100e300087834b0008044c0089844c000a054d0050
:100e40008d06e90084827200850273004c3add0051
:100e5000850272000100320015002000443ade00d5
:100e60001400b2004538de00cb45dd000b007000f9
:100e7000c540de00cb4ddd008b8070004549de00b3
:100e8000cb55dd000b017100c551de000d0378006c
:100e90002d03070003f0a1000cf0a70003f0a00051
:100ea000240337001b18b800850240000683480061
:100eb000e0834b0060044c00070037001b18b800ab
:100ec0000603400087834800faff37001b18b8006c
:100ed0008703400008844800e0844c0060054d0012
:100ee000000006001b18b800080440008984480070
:100ef000faff37000108a3000b033a005800be00b8
:100f00005801be00e3ff37000008a30006033a00c3
:100f100009047800f9ff37008103780074ff0700a7
:100f20000001be006000b8000478a30013003a007e
:100f30006220e10015003e000d0039008301d10060
:100f40000281d3008180d3008301d1000281d300cc
:100f50008180d3008301d1000281d3008180d3003e
:100f60000538b000c42add00f300b20083817200ae
:100f700007f0a70003f0a00000000600f3ff270021
:100f8000f2ff2f006110b900fbff370003ff2700bd
:100f9000f7ff37008f1fd100170307008f87e90085
:100fa0000000e00000000600801feb0012030700b5
:100fb0008f87e9000000e000000006001400fa003e
:100fc000889fbe008a9fbe008c9fbe000004be00aa
:100fd0000205be00680047000a90be000890be00ef
:100fe0002e0307000070a7000bf0a1009e099000df
:100ff0000e099000fe0090006e0090009e0290008e
:1010000034432000848252000a00320010003c0069
:10101000b4fc2f000428e1001f0034008301d1003c
:101020000281d3008180d3000080d3008502e800d4
:10103000faff3a000b00e000be023b006000100027
:10104000e080180060011900e0811900b902370042
:10105000b40020000428e10007003d00000040002b
:101060008180480002014900838149008502e9002e
:10107000faff3a00efff3700f3ff2700f2ff2f00df
:101080006110b9000b00e000aa023b000300280039
:1010900002002000010037006011b8006000b800b5
:1010a000a4023700889fbe008a9fbe000305780017
:1010b0000300e000050035000b003c0000827000da
:1010c0000402710030003200070037006000100099
:1010d000e080180060011900e081190002003b0067
:1010e00001f02d00280037000004be000200be0001
:1010f0006011b8006b092000950220000182cf002a
:101100000a0039000541b1000082cf000700390014
:101110000541b1000982cf00040039000541b1004a
:101120000882cf00010039000541b100054252009c
:10113000120032000a003b008281710061016400ec
:101140008100d1000080d3008984d3000884d300bb
:101150008b05e8000442e800f7ff3a00070037007b
:101160000804440089844c00000048008180480045
:101170008b05e9000442e900f9ff3a0083fe07000d
:101180000af0a70001f0a0004f05be004f04be000a
:1011900000000600e80207000509780000000600cc
:1011a000809feb00940207008f87e9000000e000b9
:1011b000000006002800fa00889fbe008a9fbe003b
:1011c0008c9fbe0007067800878669000c003b00f4
:1011d000030478008704780008f0a10009f0a1005a
:1011e000840f5000858f5800860f5900890f5c00ce
:1011f000030033000cf0a20001003a000cf0a10043
:10120000380207006400e1005f0032007801470007
:101210006408e100610032006c01470074855700ea
:101220003200be001201be003a04be001a05be0024
:101230001e039000be0a90008503530006003d0087
:101240000004fd008104fd000205fd008305fd0092
:101250008703ea00050378000df8a30004003200bc
:1012600060041400e0841c0060051d00e0851d0082
:101270006022b8007d0320000d38e1008006eb00fd
:101280000b0039004433dd00f300b200830173002a
:1012900039003700848272000d027800e106640094
:1012a0008b85d1000a85d3008984d3000884d300bc
:1012b0008703e900f7ff3b000800400089804800f1
:1012c0000a0149008b81490004003b0060001000c6
:1012d000e080180060011900e08119000358a300a4
:1012e000090032008d827200848272006102600007
:1012f0008301d1000281d3008180d3000080d3001c
:101300000603e8001b0037000348a30017003a005b
:101310000600e000170034000603e9000d00a300fa
:101320000000480081804800020149008381490093
:101330000348a3000f003a000600e0000900340053
:101340000603e900000040008180480002014900d6
:101350008381490001003a000003eb000348a30029
:10136000f5ff32006022b80002003700848272006c
:1013700061826600f401070003f0a1000cf0a700f1
:1013800003f0a000eb013700640147006408e100ae
:1013900002003a000df8a300e3013a003200be005b
:1013a0001201be00e30137001400fa00889fbe005e
:1013b0008a9fbe008c9fbe000004be000205be00d6
:1013c000680047000a90be000890be003302070084
:1013d0000070a7000bf0a1000bf8a30020003a005a
:1013e0009e0990000e099000fe0090006e00900093
:1013f0009e0290003443200084825200cd013200ce
:101400000a003c00b4fc2f000428e1001400340062
:101410008301d1000281d3008180d3000080d300fa
:101420008502e800faff3a00c2013700b40020004c
:101430000428e10007003c000000400081804800d3
:1014400002014900838149008502e900faff3a0060
:10145000b801370003002800020020000100370017
:101460006011b8006000b800b20137002800fa002f
:10147000889fbe008a9fbe008c9fbe0003866b00c3
:10148000980107006400e100440032006408e100b4
:101490004a0032006100e100460032006108e100cc
:1014a00049003200ec0647006000b8003d02be0073
:1014b0003d03be00f48657006011b8003d04be0035
:1014c0003d05be007d0320000b0037000000a0009a
:1014d0008d06e900130032000402420085824a00b2
:1014e00006034b0087834b000000400081804800ca
:1014f00002014900838149000802520089825a0092
:101500000a035b008b835b00f0ff3b000802420094
:1015100089824a000a034b008b834b008d06e90049
:10152000edff3a008482720086827200f707b200f3
:101530008782720001003200150020001e04900016
:101540003e0b900006035400e63fb0000368a30082
:10155000070032000000a7000500a0008301d100b1
:101560000281d3008180d3000080d3000603e8000d
:101570008301d1000281d3008180d3000080d30099
:101580000002eb000482d2006f01070003f0a1000b
:101590000cf0a70003f0a0006601370064024700ca
:1015a0006408e100600132003400be003401be0076
:1015b000f6ff37006108e1005b0132006011b800fe
:1015c0006000b800f1ff370003ff27000200200091
:1015d000fbff3700889fbe00830478000300e00013
:1015e0002c00350003003c000082700004027100f2
:1015f0002600320036432000c50020008383cf0040
:101600000a0039000541b1008283cf00070039008c
:101610000541b1008183cf00040039000541b100cc
:101620008083cf00010039000541b10085c353001c
:101630006022b800120032000a003b00848272006f
:10164000610260008301d1000281d3008180d30058
:101650000080d3000603e8008743e800f7ff3a0064
:101660000700370000004000818048000201490067
:10167000838149000603e9008743e900f9ff3a0046
:101680003101070009f0a70003f0a0004f04be00dd
:101690000000060060001000e080180060011900e2
:1016a000e0811900d3ff3b00033e2c00f7ff370019
:1016b00007f0a200bffe3700881f78000004780002
:1016c0005001be004000be0004004000858048007c
:1016d0000601490087814900009cbe000294be00bb
:1016e0000400e1000588e1000690e1000798e100b0
:1016f00002003100680044001008e8004f04780040
:1017000000000600f4874700889fbe008a9fbe0045
:101710008c9fbe008e1f78000205be000004be0034
:10172000d4b79f00e5b79f00f6b79f0087bf9f0023
:101730000000eb00c0b79f00b0b79f00a0b79f00ac
:1017400090b79f0080b79f000d042000bfb09700a6
:101750004fb09700000140000000e0000f003d0086
:101760004f08de0000007100c0b79f009e00070018
:1017700001003d0012002000a100070001003d0013
:1017800012002000a6000700b1000700b600070005
:101790000f004000c8ff0700220037004f08de009e
:1017a00000067100ccb79f008f00070001003d00cc
:1017b000120020009200070001003d0012002000ee
:1017c00097000700a20007000fb297009fb2970092
:1017d0002fb39700bfb39700a90007000000520085
:1017e00081805a0002015b0083815b0080b79f000b
:1017f00091b79f00a2b79f00b3b79f000007eb000f
:101800009f0007000020e10001a8e10002b0e10014
:1018100003b8e100010031001e0020000e00560058
:10182000c0b79f004fb297000400e00007003500ea
:1018300010002000010020006011b80008047000b2
:10184000898470000a0571008b8571008d06e9009e
:10185000beff3a000400e00003003d0082000700e4
:101860000f00400094ff07004fa897000000e00021
:1018700004003a000fb497009fb497002fb597006b
:10188000bfb59700940007004f0778004f06be00d1
:101890004f05be004f04be004f01b100000006001e
:1018a000881f780018002000881f780095ff070027
:1018b0008f87e9004f04780000000600801feb00ce
:1018c00090ff07008f87e90000000600889fbe0098
:1018d0008a9fbe008c1f78006e00070007003d0045
:1018e00073000700e00f5b00e08f5b0007003d0026
:1018f000320007000006eb00040037003400070048
:1019000002003d002a0007001c00200072000700b2
:10191000e3ff07000203be000002be000c00e0006f
:1019200001003200220007000400be000601be00d4
:101930004f0678004f05be004f04be0000000600b1
:10194000889fbe008a9fbe008c1f78005100070050
:1019500005003d0056000700e00f5b00e08f5b00d4
:1019600006003d00040037001900070003003d0099
:101970006000b8006011b8001000070056000700b2
:10198000ceff07000203be000002be000c00e00014
:1019900001003200060007000400be000601be0080
:1019a0004f0678004f05be004f04be000000060041
:1019b0006000b8006011b800000037000402500059
:1019c00085825800060359008783590000000600ed
:1019d0000006eb00e00f5200e08f5a00e00f5b00c2
:1019e000e08f5b00000006000180400090b79f0080
:1019f0000001eb008fb097000100e000000006003e
:101a00000200700090b79f000180400080b79f00e7
:101a10000001eb00ffa897000100e00000000600b5
:101a20000200700080b79f00018040006faa9700fd
:101a3000cf20de0001007000f0af9f0004024200e2
:101a4000250007004f18de000002720000000600ab
:101a5000e4af9f000804440089844c000a054d004f
:101a60008b854d00000006003fb29700cfb2970073
:101a70005fb39700efb3970000fe2f000000060051
:101a80003fb09700cfb097005fb19700efb19700dc
:101a9000000006000205be000004be00e00f50007a
:101aa000e08f5800e00f5900e08f59000000060059
:101ab0006000b8006011b800080450008984580024
:101ac0000a0559008b8559001c002000e00f5200c8
:101ad000e08f5a00000006000800be000a01be00a8
:101ae00000000600680447000294be000094be0097
:101af000fc0447008694be008494be000900780070
:101b0000660007000800780064000700990078006c
:101b1000814f70000b003b000800be0093000700df
:101b20004f00b10003003700f3ff2700f2ff2f0042
:101b30006110b9004f06be004f05be004f04be0045
:101b40000080fa0000000600180020005700200066
:101b5000080453000d003d000600200097fc2f00f4
:101b60000740e1001e0034008482720061026000c0
:101b70008301d1000281d3008180d3000080d30093
:101b80000804e800f8ff3a00470020006104600004
:101b900005047400040464000d003200610040007c
:101ba000e080480060014900e081490003b8a500d9
:101bb000070032000603e8006538e10004003a003f
:101bc0008301d1000281d3008180d3000080d30043
:101bd000f87f20000830e10003003500080378009a
:101be0006000b8006011b8004433dd00f300b200bb
:101bf0008301730000000600889fbe008a9fbe001c
:101c00008c9fbe000404be000605be00809fbe007f
:101c1000829fbe0063000700040678000800be0033
:101c20000a01be005f000700840678004f03be0073
:101c30004f02be008d4f76007fb097001300330037
:101c4000f0ff2f008b8f6b0006003b000d06660037
:101c50000c00a7000a00370007f0a60010002000c3
:101c60000a003700880f5200898f5a008a0f5b00e4
:101c70008b8f5b00030039001000200001003e0044
:101c80000000200007f0a7000000ea004f06be0099
:101c90004f05be004f04be00000006008000780023
:101ca0005002be005003be004439de00f700b2000f
:101cb000f37f200003016100090032000218e100f7
:101cc00016003a008501720083017300838173005e
:101cd0000008200015003a004000200013003700e3
:101ce00085017200830173008381730005003a004f
:101cf00004a8be0006a8be00100020000b0037009c
:101d00000201e9000402420085824a0006034b00fa
:101d100087834b000748a300f9ff32000740a0006b
:101d200004a8be0006a8be00200020008000980085
:101d300092009800000006000003be00ecfb0700c4
:101d40006220e100020032000600be00050005002e
:101d5000e507b100f107b20004f0230084807000b1
:101d600007f0a70001f0a00024000500e482400075
:101d70001078a30007003200640240001178a3002d
:101d80003400be001401be00040032000330a7007e
:101d9000000006003500be001501be000330a000a3
:101da0000000060005ff27000582610007003200e1
:101db0000428e100010032002400050006000700ad
:101dc00001003a0044000500040805000200070075
:101dd000f9ff3a00140005006f8261008102700073
:101de0008502710085027200000006000c00fa00f6
:101df000889fbe0000047800cfb09700f0ff270056
:101e0000d0bf9f008004eb0099bf9f0088bf9f0058
:101e1000a8bf9f00200c2000b0bf9f007881570012
:101e200070805700890007000fb8970009487800b4
:101e30000fb8970008045000080078004f04be0057
:101e40000080fa00000006000001780000c2b30024
:101e5000010037000201e8009240780080cf500076
:101e6000fcff3200e9cf5000faff3200d0c2b300cd
:101e700080cf500003003a000201e80014c0b30014
:101e8000050037000042eb00b0c2b30080cf500025
:101e900001003a000201e8008000eb0005fd2f0080
:101ea000040037006a08b900008041008500400046
:101eb0000201e8009201fb0005804100e90f50009b
:101ec000f8ff36000404e000010032008100ea005f
:101ed0000100780000000600800078003004e00077
:101ee000feff3a00010050000000e900000006007b
:101ef000889fbe008a1f7800804078000004e000c0
:101f000021003d008040ea00d0c6b30080cf5000e1
:101f1000090034008104fb00420620001100090082
:101f20008204d80000017800010078004311dd0030
:101f30002ab920001f0037000100fb0023b9200050
:101f400039003700a2002000110009000200d8006b
:101f500000017800010078004311dd000301410019
:101f60004300dd00030040003002be002003be003d
:101f700042209000d2209000f22190006221900037
:101f800070fb07002e003700d0c6b30080cf500092
:101f9000230034008104fb004206200011000900e8
:101fa0008204d80000017800010078004311dd00b0
:101fb0002ac420000a014100a800200011000900e5
:101fc0000800d8004300dd000a00400040229000d5
:101fd000d022900060239000f023900002889000af
:101fe00092889000b28990002289900055fb0700ea
:101ff000801f780001027800110009008804d800d1
:102000000102fd004f0078000402fb004322dd00c6
:102010000a0242005403be004402be00d8ff37004b
:102020000100fb0023c42000eacf5000c5ff3c00a4
:102030004300dd00030040005001be004000be0030
:102040004f0578004f04be00000006008f03b0006b
:10205000889fbe008a9fbe008c9fbe008e1f7800a6
:10206000e0b79f00f1b79f0082bf9f000000eb0028
:10207000a0b79f003b0537008001eb0050c2b300c2
:1020800080cf5000090032000100fb00efb0970044
:1020900041050700e10f400032053200afb0970064
:1020a0008100e800a1b79f002e0537007fb197009f
:1020b00092407800b0c2b30080cf500019003200c7
:1020c00007003c006b40500080cf500010003200f1
:1020d0006340400080cf500021003a0016003700d6
:1020e000d0c2b30080cf50000400320063404000f3
:1020f00080cf50001a003a00140037000330a000cf
:102100007fb297000402e800f4b79f00e7ff3700b2
:102110000300a000ffb297008502e800f5b79f001a
:10212000e2ff37000310a0007fb697000c06e8001e
:10213000fcb79f00ddff370003b0a0007fb0970021
:102140000000e800f0b79f00d8ff37000320a00090
:10215000ffb097008100e800f1b79f00d3ff370080
:102160000318a300010032000300a1000338a300fc
:10217000010032000320a1000100fb0002fd2f003e
:1021800002004000e90f500010003e000002eb008a
:1021900094a79f00020278009fa297006a28b900c6
:1021a0007fb697001c01fb000001410004014100c3
:1021b00092a79f005c00fb00fcb79f00040040005a
:1021c000e90f50000d003e00f3ff37000000eb0068
:1021d00090a79f00a0c2b30080cf500007003a0034
:1021e0008fb897004101780081bf9f0092a79f00a0
:1021f0007fb297000402e800f4b79f00e0c2b3008a
:10220000ffb29700954f100021003a008306780036
:102210000de0a0008500e80064405000914f1000e0
:1022200004003200f1b79f000006eb00bcb79f002e
:10223000100037000fb89700c000780080bf9f00e3
:10224000b1b79f007fb197000281e800f2b79f000d
:10225000130037003fb297006a20b9000000410028
:1022600003004000b0b79f00ffb297008502e8006e
:10227000f5b79f007fb697001c01fb0003fd2f0000
:1022800003004100e90f5000f2ff36000400370060
:10229000830678000dc0a0000000eb00b0b79f00df
:1022a0007fb19700b2407800f2b79f00c17f9f00d6
:1022b000c0c6b30080cf50002700320014003c009d
:1022c0006840500080cf50009d00320009003c0063
:1022d0006c40500080cf5000290032006b4040001d
:1022e00080cf5000720032000104e000a3043200ed
:1022f0008e00370060c6b30080cf50001c00320053
:102300006340400080cf500088003a008c003700c6
:1023100030c7b30080cf50001c00320007003c00e3
:102320006440500080cf5000130032000040e800ad
:1023300080cf50007d003a001100370050c7b30035
:1023400080cf50007d0032006340400080cf5000bd
:1023500076003a000b003700000028000d48a3006b
:1023600001003a000001200080867600ccff370093
:102370000da0a000720037000d60a00070003700b3
:102380000d50a0000d70a0006d0037008fb99700b0
:102390004300780083bf9f00000478000000e00045
:1023a00001003a0028cf20008004eb000100370034
:1023b0008104e80089007800088044001004e000ef
:1023c000fbff3a003fb297000400e0000300320038
:1023d000890f520001003100840478000007eb00ef
:1023e0009fa29700898f5200010036000987520092
:1023f0004368de00e106600019003a000d0678002f
:1024000009003700efb097000002200062040700c7
:10241000e10f4000030032002fb097000000e800f9
:10242000a0b79f000c06e8008e0f5600f5ff3a009b
:102430000087eb000a003700880078003100fb00bd
:1024400001047800efb0970053040700e10f40004b
:1024500003003200afb097008100e800a1b79f00f1
:102460000900e90080047800e10f4000f2ff3a0023
:102470000006eb000d00e0000a003a0039043700c6
:10248000efb097000002200043040700e10f400076
:10249000030032002fb197000201e800a2b79f00ad
:1024a0000c06e8008e0f5600f5ff3a002d043700a9
:1024b0008fb997004300780083bf9f00cf80de0074
:1024c00001017800820178000205be000004be0010
:1024d0000203be000002be004822de00482edd00de
:1024e00004027600c47f9f000d48a3000a0032005a
:1024f0000404e00008003200e14f42000600320010
:10250000d1fb2f000f80400004487800184098004d
:102510002900200002003700d07f9f001900200012
:10252000d2fb2f000f044100a6ff3700c3fb2f0092
:102530000f84410019002000a2ff37000d0cb300ea
:102540000070200000826600310232000dc8a30036
:102550000200320064002000b4b79f000d48a300c1
:10256000050032000fba97004401be004400be00cf
:1025700084bf9f00040037008fba97004500be005b
:1025800085bf9f0064fa0700e0af9f00f1af9f0096
:1025900082b79f0093b79f006022b8006033b800f5
:1025a0006fa89700ffa897000fb197009fb1970001
:1025b00078fa07000000e0000a003d006fa89700cd
:1025c000ffa897000fb197009fb1970003f0a200fa
:1025d000e0af9f00f1af9f0082b79f0093b79f00cd
:1025e0003d00b3000000eb0080a79f006022b80010
:1025f0006033b8006fa89700ffa897000fb197004d
:102600009fb1970068fa07000000e0003500320033
:102610006fa89700ffa897000fb197009fb1970090
:1026200066fa07009ffa070003fc2f000f814100a4
:10263000d8fa07000fa097000000e9006300b90076
:10264000a2002000110009000200d8008000fd0057
:1026500081a79f000100e00002003d000100e900a9
:1026600080a79f000fa497000840ea0020fe070003
:102670006faa9700ffaa97000fb397009fb3970028
:10268000b0f90700a0af9f00b1af9f00c2af9f009d
:10269000d3af9f006022b8000600200007ff230090
:1026a0003cfa07000000e00002003d000800e900dd
:1026b0000b0037006022b80006002000470224000b
:1026c0002fa89700bfa897004fa99700dfa99700f0
:1026d000b3fa07000000e000020035000800e8003f
:1026e00080a79f003fb29700f80f520057003c00b0
:1026f000d0c6b300804f5200290036000485fb008d
:1027000042062000110009000285d800000178006f
:10271000010478004311dd002bb920000b014100ba
:102720006022b8000600200007fe23000288900007
:1027300092889000b28990002289900081f9070068
:10274000a9002000809fbe00110009000984d80064
:10275000000478004f00be004344dd000b04440039
:1027600048229000d822900068239000f82390001f
:1027700074f90700801f7800010278001100090039
:102780000985d8000102fd004f0078004322dd00da
:102790000b0242005403be004402be001f0037007b
:1027a0000480fb0029b92000ea4f520014003600d3
:1027b000a2002000110009000280d800000178006a
:1027c000010478004311dd00090141006022b800d6
:1027d0000600200007fe230042209000d220900037
:1027e000f22190006221900056f907004344dd0079
:1027f000090444003802be002803be000700370069
:102800004300dd00090040006022b80006002000ff
:1028100007fe23005001be004000be0049f907003a
:102820000002be000203be006fa89700ffa8970039
:102830000fb197009fb197005efa0700e0af9f00cd
:10284000f1af9f0082b79f0093b79f000fa497003e
:10285000e90f540015003c006022b8006033b80056
:102860006fa89700ffa897000fb197009fb197003e
:10287000cdf907000000e000320032006fa8970099
:10288000ffa897000fb197009fb19700c6fa070005
:10289000e00f5000e08f5800e00f5900e08f590022
:1028a00028003a00e10f5400260034000400200004
:1028b00005002e00b6e02200170124002fa8970083
:1028c000bfa897004fa99700dfa99700b1f90700ab
:1028d0000000e00002003d007300540001003700da
:1028e0007200540080a79f000fc0970080fd070072
:1028f000a0af9f00b1af9f00c2af9f00d3af9f00ba
:102900000002be000203be006fa89700ffa8970058
:102910000fb197009fb19700d4fa0700a2fa070001
:102920000205be000004be006000b8006011b800df
:10293000a0a79f00b1a79f00c2a79f00d3a79f0099
:102940002e0037006fa89700ffa897000fb19700df
:102950009fb1970094fa07000205be000004be0074
:10296000e00f5000e08f5800e00f5900e08f590051
:102970000200350017fb070013003700100020008d
:10298000010020006011b80008006000898060002c
:102990000a0161008b8161008b03d1000a83d3009f
:1029a0008982d3000882d300000072008180720007
:1029b000020173008381730006fb07000002be0062
:1029c0000203be00fbf907000002be000203be00c6
:1029d0006fa89700ffa897000fb197009fb19700cd
:1029e00033fb0700a0a79f00b1a79f00c2a79f00cd
:1029f000d3a79f000000eb0080a79f0014c0b30086
:102a000025af20000b0037000400fb004300dd0071
:102a1000050040005001be004000be000040e10043
:102a200001c8e10002d0e10003d8e1000300390051
:102a30000442e800f44f5200f3ff3a00c47f9f00c5
:102a40000400fb00bfb09700008040008fa09700fb
:102a5000010040001fa19700000751004b68de00f5
:102a600061006000004678000004e00003003a00c6
:102a7000bfb197000300e000010032000e07e9003b
:102a800063806600010032000e07e9000d28a300f4
:102a900026003200e18066000d18a3000c00320011
:102aa000d00220000100e00001003a000080e900af
:102ab000efb09700b8020700e10f400018003200a5
:102ac0002fb297000402e800a4b79f00140037005b
:102ad0000100e00012003200efb097000002200079
:102ae000ad020700e10f40000d003200afb29700c9
:102af0008502e800a5b79f0009003700efb09700f6
:102b000000032000a4020700e10f40000300320090
:102b10002fb097000000e800a0b79f000e07e90063
:102b20000e00e000f5ff3c003d0037000d38a3002b
:102b30000a0032000b003700efb0970000022000bf
:102b400095020700e10f400003003200afb097008c
:102b50008100e800a1b79f000e07e9000e00e00029
:102b6000f5ff3c00e18066000d18a3000c00320068
:102b7000d00220000100e00001003a000080e900de
:102b8000efb0970084020700e10f400024003200fc
:102b90002fb197000201e800a2b79f002000370084
:102ba0000100e0001e003200efb09700000220009c
:102bb00079020700e10f400019003200afb1970021
:102bc0008301e800a3b79f00150037000000fb0059
:102bd0004300dd0021af2000010040003002be00b4
:102be0002003be000800be000a01be002cfb070047
:102bf000a4002000050020006033b8002ffb070070
:102c00000003b000efb0970063020700e10f40003f
:102c1000030032002fb297000402e800a4b79f001f
:102c2000cf7a97000540e900c07f9f00e14f400048
:102c3000e6ff3a000b003700efb0970000032000da
:102c400055020700e10f4000030032002fb097004b
:102c50000000e800a0b79f000fa097000000e90067
:102c600080a79f000fa097000000e000f2ff3c004b
:102c7000bfb09700f28f50000300340020c1b300b2
:102c8000c07f9f00020037006fe19700c27f9f0066
:102c9000cf7897000100fb00bfb197000080510082
:102ca000e0a79f000104e00002003a000c04e000ed
:102cb00008003200efb09700e00220003602070063
:102cc000e10f4000030032002fb297000402e80039
:102cd000a4b79f004f78970085fc07000002be0054
:102ce0000203be002fa09700bfa097004fa197003e
:102cf000dfa1970013f80700abf907001e003700ab
:102d00000000fb004300dd002caf20000c00400061
:102d10003002be002003be000800be000a01be0053
:102d2000dffa0700a4002000050020006033b8008f
:102d3000e2fa07000003b000efb0970016020700a8
:102d4000e10f400003003200afb297008502e800b7
:102d5000a5b79f00cf7897000100fb004300dd007e
:102d60000c0040003002be002003be000800be0080
:102d70000a01be00d1fa07000205be000004be0031
:102d80004f7997000240e900c07f9f00e14f40006b
:102d9000dbff3a000006eb0009003700efb09700b8
:102da00000032000fc010700e10f40000300320097
:102db000afb197008301e800a3b79f000c06e800bd
:102dc0006fa29700840f5600f4ff3a000d38a3005d
:102dd000e40132000e00e000e20134000006eb00e6
:102de000efb0970000022000eb010700e10f400068
:102df00003003200afb297008502e800a5b79f003c
:102e00000c06e8008e0f5600d6013200f4ff3700a2
:102e10000d007800000cb20028003a000d00e00020
:102e200005003d000fbe97004c05be004c04be00df
:102e30008cbf9f00140037000d48a3000b00320028
:102e40000fb997004200be0082bf9f004f89de008d
:102e5000cf91de000002be000203780082037800fa
:102e60000605be000404be00070037008fb99700b6
:102e70004300780083bf9f0000047800cfc4de00c9
:102e8000090578008a057800e00f5400e08f5c00a7
:102e9000e00f5d00e08f5d0020003d003d00b300cd
:102ea0006000b8006011b800080450008984580020
:102eb0000a0559008b855900180037000d00e00005
:102ec00005003d000fba97004405be004404be0053
:102ed00084bf9f00110037000d48a3000800320096
:102ee0008fba97004500be0085bf9f00040178009f
:102ef000840178000205be000004be000700370010
:102f00000fbe97004c0078008cbf9f000004780033
:102f1000090020000a0020000b0020003fb09700ad
:102f20000000e00007003a00e00f5400e08f5c0072
:102f3000e00f5d00e08f5d0002003a00110020000c
:102f4000b1b79f000d017800020cb200d2b79f000c
:102f500000042000800f51002d00320003003c00cf
:102f60000200e000080032003a00370000082000ac
:102f7000dfb19700808f510014003200000c200058
:102f8000808f510033003a0014c0b30025af2000f9
:102f90000b0037000400fb004300dd00050040008b
:102fa0005001be004000be000040e10001c8e10049
:102fb00002d0e10003d8e100250039000442e80016
:102fc000f44f5200f3ff3a002100370014c0b30061
:102fd00025a720000b0037000400fb004300dd00a4
:102fe000050040005001be004000be000040e1006e
:102ff00001c8e10002d0e10003d8e100140039006b
:103000000442e800f04f5200f3ff3a00100037008e
:1030100014c0b300259c20000b0037000400fb0007
:103020004300dd00050040005001be004000be002e
:103030000040e10001c8e10002d0e10003d8e10056
:10304000030039000442e800f64f5200f3ff3a0053
:10305000c47f9f004f7a97000400fb00bfb2970027
:10306000850f500002003d00c57f9f00040037001f
:103070003fb69700800f560001003d00b0b79f009b
:103080001fa097000000e00005003200638066008a
:10309000030032009fa097008100e90091a79f00e4
:1030a0000de8a3000b0032001fa19700bfb19700ed
:1030b000830f510003003c000002eb0094a79f0027
:1030c000040037009fa297003fb697008c82520001
:1030d00095a79f00408c200000806600018420009e
:1030e000810f500006003a001fa097000000e0008a
:1030f000110032000000e90090a79f000e00370089
:10310000008c20000080660001882000810f5000a4
:1031100009003a009fa09700e28f500003003c0096
:103120000001eb0092a79f00030037009fa19700ca
:103130008381e90093a79f004f7a97000400fb006a
:103140008002eb00c5b79f001fa69700800f5600b6
:103150000200340000005600c0b79f000d28a300f5
:1031600052003200e18066000d18a3000c0032000e
:10317000d00220000100e00001003a000080e900d8
:10318000efb0970004010700e10f40002700320074
:103190002fb097000000e800a0b79f002300370081
:1031a0000100e00009003200efb0970000022000ab
:1031b000f9000700e10f40001c003200afb097009b
:1031c0008100e800a1b79f0018003700008c2000a4
:1031d0000080660001882000810f500013003a0033
:1031e000efb0970000032000eb000700e10f400064
:1031f000030032002fb197000201e800a2b79f0040
:10320000800520000d58a30001003a00800720002f
:10321000efb09700e0000700e10f4000030032002c
:10322000afb197008301e800a3b79f004fb29700aa
:103230000400e0000f0032000006eb00efb0970042
:1032400000032000d4000700e10f4000030032001b
:10325000afb297008502e800a5b79f000c06e80012
:103260004fb09700800f5600f4ff3a008000eb004b
:10327000c1b79f003fb197008200e900c308dd009d
:1032800020af20000080400080af9f0020a72000da
:1032900000804000f0a79f00209c20000087400095
:1032a0008001eb0093af9f00980037004fb297006a
:1032b0000400e00011003200688066000f003a0050
:1032c00000067800efb0970000022000b20007006f
:1032d000e10f400003003200afb297008502e80022
:1032e000a5b79f000c06e8004fb09700800f56006e
:1032f000f4ff3a008000eb00c1b79f00e180660058
:103300000d18a3000c003200d00220000100e000e4
:1033100001003a000080e900efb097009e0007002e
:10332000e10f40000e0032002fb197000201e800cb
:10333000a2b79f000a0037000100e0000800320039
:10334000efb097000002200093000700e10f40005b
:1033500003003200afb197008301e800a3b79f00dc
:10336000008c20008080660000842000808f500048
:1033700009003a00efb09700000320008600070024
:10338000e10f4000bbff32002fb297000402e800bb
:10339000a4b79f00b7ff370000882000808f50003f
:1033a000b4ff3a00efb09700000320007a00070056
:1033b000e10f400003003200afb297008502e80041
:1033c000a5b79f00800520000d58a30001003a001a
:1033d00080072000efb097006f000700e10f40006a
:1033e000a4ff32002fb697000c06e800acb79f0090
:1033f000a0ff370000042000dfb09700808f50004e
:103400002700320003003c000100e0000800320009
:103410002b003700000820005fb19700800f51009b
:1034200011003200000c2000800f510024003a00ef
:103430008fa997003302be002303be000800be0020
:103440000a01be0016f90700a400200005002000b4
:103450006033b80019f9070004c3b3000442400008
:10346000c47f9f00160037009ccf20000d58a3009a
:1034700001003a00acd020007fa097003002be00cf
:103480002003be000800be000a01be0004f90700c8
:103490006f0060006c467800cc7f9f00080037000a
:1034a0003e02be002e03be000800be000a01be00a0
:1034b000fbf80700674060000043b000c07f9f003a
:1034c000cf7897000100fb00efb0970032000700b3
:1034d000e10f4000030032002fb197000201e80025
:1034e000a2b79f009fa997008301e80093af9f00b8
:1034f0000faa97006802520084af9f00ffa29700b6
:10350000e8825200f5a79f00680757001fae97009a
:103510003fb09700800f5600b6ff3a000d38a30069
:1035200010003200cfb097000100e0000d00340021
:103530000006eb00efb09700000220001600070025
:10354000e10f4000030032002fb197000201e800b4
:10355000a2b79f000c06e800cfb19700830f56007a
:10356000f4ff3a007fb29700b4407800f4b79f00b0
:10357000c17f9f000104e000bffa3a002fb097001e
:103580004f0778004f06be004f05be004f04be0037
:103590008f03b10000000600889fbe000001780084
:1035a00001047800b10090000118a3003d00320032
:1035b0000198a30003003a00180090000000e0000a
:1035c00038003a000190a00031049800820478008d
:1035d000f90fb200180090000000e00002003a006d
:1035e00028009000000c78003800900000b8a3007c
:1035f0000600320000a8a3000400320021002000d1
:103600006011b8000800780049000700b800900079
:103610000100780000b0a10030049800ea8f540047
:1036200005003a000178a30003003a008800780002
:10363000d0002000d8ff07009800900058009000ac
:10364000808f50000b0032000100e8001004980049
:103650001800780009587800000c780011c0b300f9
:10366000c0d1200001487800ea8f540006003200e3
:103670000f0037008800780009407800c600070076
:10368000800478000a003700380090000088a3000a
:10369000060032000800780095000700e10f4000a6
:1036a00002003a008084eb0001003700a9002000ee
:1036b000090078004f04be0000000600881f780053
:1036c0000004780040009000110020006011b80054
:1036d0009ff307000001be00180090000000e0000a
:1036e00002003d000000eb0010049800280090004c
:1036f0000000e00008003200380090000098a300ad
:103700000500320018009000cf80de00020040006b
:10371000838048000400370018009000cf80de004e
:1037200000005100818059004f047800000006001d
:103730000400fa00889fbe008a9fbe008c1f78009c
:103740000006780092bf9f00a3bf9f00010478008d
:10375000300090000040a100300698002c0090003e
:103760000000e00006003a004c00900078f30700eb
:10377000e10f4000e08f480057003a005400370046
:10378000e18f500005003200e28f50000c00320043
:103790000100e000200032004d0037000c007800ee
:1037a000c6ff07001fb99700afb99700020140009c
:1037b0008381480092bf9f00a3bf9f00160037007f
:1037c0000c0078004a0007004c0090001100200017
:1037d0006011b8005ef307000005be004c009000c9
:1037e000880078006011b80059f307000004be009b
:1037f0004c0090008000eb000a01be0054f307006b
:103800001fba9700afba97000402440085824c00ab
:1038100094bf9f00a5bf9f000c007800a7ff070082
:103820001fba9700afba97000001520081815a0079
:10383000030032003c00900000b0a0003006980069
:103840003c0290000408a3000f00320062036200f3
:103850000d003a00e00f5100e08f59000a003500da
:103860009c0290006128b900800f5100818f59009f
:1038700005003c0002805200100698001c0e41001a
:1038800006007800150037000498a30005003200f8
:103890001c0090000000e000020032000c007800e4
:1038a000130007008000eb0011069800ac029000a6
:1038b000050e78004c0090001fb99700afb9970033
:1038c00023f30700e00f5000e08f580002003d0096
:1038d0000080eb00010037000000eb004f0678008d
:1038e0004f05be004f04be000080fa000000060035
:1038f000881f780000047800300090000008a300c2
:1039000007003200800078000120b20004003a0075
:1039100011049800a8009000010c780017003700ef
:103920000018a300190032000098a300170032000d
:10393000a80090000100e00014003200180190007f
:103940000200e00011003200480090000df3070073
:1039500098009000810f5000030032003800900062
:103960000003b300300498000000eb00100498003e
:1039700028009000000c7800380090000058a30048
:10398000020032000080eb00010037000000eb0075
:103990004f047800000006000200fa00889fbe0075
:1039a000a0ff9f000104780031009000e200600059
:1039b00004003a000003b30030049800110498009a
:1039c00018003700d80490000900e0001a003a00ff
:1039d0006c00600004003a003300070020049800e7
:1039e000e10f400011003a002904980059049800a2
:1039f000380090000020a0003004980019049800be
:103a00004800900012002000e6805700ddf2070019
:103a1000e10f50001f003200380090000003b30097
:103a2000300498000080eb001c00370000202000cc
:103a3000500498000a00370018019000a800900078
:103a400048009000cff2070098009000810f5000ce
:103a500003003200380090000003b30030049800e7
:103a6000100020001004980028009000aff8970084
:103a70000148780028009000000ce800b800900091
:103a80000080eb000158a30004003a000190a00060
:103a900031049800aff897000180fb004f04be008e
:103aa0000080fa0000000600f16880000100e000dc
:103ab0000300320011007800f0688800030037002e
:103ac00000202000e6f2070080007800e18f40002f
:103ad00002003a00906e260000698800010078001c
:103ae00000000600f168800001087800f068880096
:043af00000000600cc
:020000040000fa
:020000040001f9
:0457f800bdfa0000f6
:020000040000fa
:020000040001f9
:0457fc007f3e0000ec
:020000040000fa
:10000800002d0000002d0000002d0000002d000034
:10001800002d0000002d0000002d0000002d000024
:10002800002d0000002d0000002d0000002d000014
:10003800002d0000002d0000002d0000002d000004
:10004800002d0000002d0000002d000000280000f9
:10005800e8270000002d0000002d0000002d000002
:10006800002d0000002d0000002d0000002d0000d4
:10007800002d0000002d0000002d0000002d0000c4
:10008800002d0000002d0000002d0000002d0000b4
:10009800002d0000002d0000562800003e2800001a
:1000a800002d0000002d0000002d0000002d000094
:1000b800002d0000002d0000002d0000002d000084
:1000c800002d0000002d0000002d0000002d000074
:1000d800002d0000002d0000002d0000002d000064
:1000e800002d0000002d0000002d0000002d000054
:1000f800002d0000002d0000002d0000002d000044
:10010800002d0000002d0000002d0000002d000033
:10011800002d0000002d0000002d0000002d000023
:10012800002d0000002d0000002d0000002d000013
:10013800002d0000002d0000002d0000002d000003
:10014800002d0000002d0000002d0000002d0000f3
:10015800002d0000002d0000002d0000002d0000e3
:10016800002d0000002d0000002d0000002d0000d3
:10017800002d0000002d0000002d0000002d0000c3
:10018800002d0000002d0000002d0000002d0000b3
:10019800002d0000002d0000002d0000002d0000a3
:1001a800002d0000002d0000002d0000002d000093
:1001b800002d0000002d0000002d0000002d000083
:1001c800002d0000002d0000002d0000002d000073
:1001d800002d0000002d0000002d0000002d000063
:1001e800002d0000002d0000002d0000002d000053
:0801f800002d0000002d0000a5
:020000040000fa
:10020800002d0000002d0000002d0000002d000032
:10021800002d0000002d0000002d0000002d000022
:10022800002d0000002d0000002d0000002d000012
:10023800002d0000002d0000002d0000002d000002
:10024800002d0000002d0000002d000000280000f7
:10025800e8270000002d0000002d0000002d000000
:10026800002d0000002d0000002d0000002d0000d2
:10027800002d0000002d0000002d0000002d0000c2
:10028800002d0000002d0000002d0000002d0000b2
:10029800002d0000002d0000562800003e28000018
:1002a800002d0000002d0000002d0000002d000092
:1002b800002d0000002d0000002d0000002d000082
:1002c800002d0000002d0000002d0000002d000072
:1002d800002d0000002d0000002d0000002d000062
:1002e800002d0000002d0000002d0000002d000052
:1002f800002d0000002d0000002d0000002d000042
:10030800002d0000002d0000002d0000002d000031
:10031800002d0000002d0000002d0000002d000021
:10032800002d0000002d0000002d0000002d000011
:10033800002d0000002d0000002d0000002d000001
:10034800002d0000002d0000002d0000002d0000f1
:10035800002d0000002d0000002d0000002d0000e1
:10036800002d0000002d0000002d0000002d0000d1
:10037800002d0000002d0000002d0000002d0000c1
:10038800002d0000002d0000002d0000002d0000b1
:10039800002d0000002d0000002d0000002d0000a1
:1003a800002d0000002d0000002d0000002d000091
:1003b800002d0000002d0000002d0000002d000081
:1003c800002d0000002d0000002d0000002d000071
:1003d800002d0000002d0000002d0000002d000061
:1003e800002d0000002d0000002d0000002d000051
:0803f800002d0000002d0000a3
:020000040000fa
:103af400a44a000001a000000a0d0000436f00006a
:103b04006d7000006173000073200000436f0000bb
:103b1400756e0000746500007220000056300000cd
:103b24002e3100000a0d0000004d0000424100004b
:103b3400524900002032000030310000300a0000f9
:103b44000d0000004d4500005353000041470000a4
:103b54004520000050450000524900004f44000039
:103b64002049000053200000256900002053000074
:103b7400454300004f4e0000445300002e0d00004a
:103b84000a000000594f0000552000004841000081
:103b94005645000020200000352000005345000059
:103ba400434f00004e44000053200000544f0000d7
:103bb400204500004e54000045520000204d0000f6
:103bc400454e0000550a00000d480000495400000d
:103bd400204500004e54000045520000204e0000d5
:103be4004f5700000a0d0000004500004e5400002d
:103bf40045520000204e00004557000020500000b0
:103c040045520000494f00004420000028300000c5
:103c14002d3600003535000033350000293a000008
:103c24000050000045520000494f000044200000ad
:103c340049530000204e00004f570000202500008b
:103c44006920000053450000434f00004e4400002b
:103c5400532e00000d0a0000004900004e560000db
:103c6400414c000049440000204900004e5000002f
:103c7400555400002c200000535400004152000011
:103c8400544900004e47000020550000500d00002c
:103c94000a000000244d000042540000524e00006f
:103ca4002c250000352e0000326600002c25000073
:103cb400316900000d0a0000002400004d4200009c
:103cc400545200004e2c0000253000002e3200001b
:103cd400662c000025310000692a0000253200000e
:103ce400580d00000a000000500000005041000080
:103cf40055530000494e0000472000004f55000076
:103d040054500000555400000d0a000000520000f9
:103d14000052000045530000554d0000494e00007c
:103d2400472000004f550000545000005554000037
:083d34000d0a00000000000070
:020000040000fa
:103d3c003801fa000080eb0060198800416a20000d
:103d4c009140780000ceb30000c06000a040b300ea
:103d5c00a4e6b700b16c20009140780000ceb3000f
:103d6c0000c060003040b300cbe6b700616a2000b1
:103d7c009140780000ceb30000c06000c040b3009a
:103d8c00a6e6b700d16c20009140780000ceb300bd
:103d9c0000c060005040b300cde6b7000e03070032
:103dac00cf060700e1d7290010002000c10307004f
:103dbc0071d9290010002000be030700100020005c
:103dcc00ce06070020002000cc0607000000eb0008
:103ddc0010879800411220008e80400040cab3002a
:103dec0080487800411220008e80400090c0b300c3
:103dfc0090409800411220008e80400000cab30011
:103e0c00a0409800701220000e004000a1d729009d
:103e1c0003000900315878004000b1003000200048
:103e2c00001f980040002000701798000000eb0065
:103e3c00601798000000eb00501798000000eb0092
:103e4c00401798000000eb00301798006000b80095
:103e5c00700f9800011798006000b800500f980080
:103e6c00610f98000000200001f82b00300f980023
:103e7c00410f98000000200001f82b00100f980053
:103e8c00210f98006000b80070079800010f98008f
:103e9c001000200060079800e001200050079800f7
:103eac0040c7bf00614060000004e00005003a001c
:103ebc0040c7bf00624060000004e00001003a000f
:103ecc0009003700014e8000b0032000808f5000a5
:103edc0003003c00004e80000000e00002003c00ab
:103eec00e0012000004e8800c01220000e004000af
:103efc0088f10700004e8000410d20008e804000ac
:103f0c00801f780040da2900801f780001007800bb
:103f1c00b3f70700e4875700410d20008e80400066
:103f2c00100020006303070041dc29001000200072
:103f3c00600307006000b800008fbe001e00370051
:103f4c00001320000e00400072f107000e199100c2
:103f5c009e1991006e109100fe109100000051000e
:103f6c0081805900e0f10700008fbe0002742c0024
:103f7c00e3a524001e00be0006f20700008fbe0061
:103f8c0020002000cf030700410820008e80400055
:103f9c001200200010002000b00107000000e0001b
:103fac0005003200100020003007980000002000af
:103fbc0001122400008fbe0002002000030a24001e
:103fcc001e00be0035f207000000e000dcff3400ec
:103fdc003e009000e10f50002e003a0071df2900e6
:103fec001000200033030700270037004108200091
:103ffc008e80400012002000100020009701070066
:10400c000000e0001e003200400820000e004000be
:10401c008af70700500798005e0090000000e0004f
:10402c00120034005e019000024e8800004e8000a9
:10403c00410d20008e804000801f780030e1290067
:10404c00801f78000100780065f70700e4875700af
:10405c00410d20008e804000100020001503070049
:10406c000000eb003007980005003700f1e2290052
:10407c00100020000f0307000000eb003007980031
:10408c00200020008f0307003e009000e10f50003d
:10409c00d6ff32001000200025060700200020006b
:1040ac0023060700c01220000e00400019f1070083
:1040bc00000037004e1090000000e00013003a00a2
:1040cc001e8090000000e00010003a000000eb00a1
:1040dc002007980009003700ae00900070122000f5
:1040ec000e004000e140780020002000b9020700db
:1040fc002e0090000000e80020079800ae00900011
:10410c007e109000808f5000f3ff35004e10900011
:10411c00e10f500014003a001e8090000000e000f7
:10412c0011003a000000eb00200798000a0037004d
:10413c00ae009000401220000e00400000804000b5
:10414c009040780020002000a20207002e00900072
:10415c000000e80020079800ae0090000e189000b8
:10416c00808f5000f2ff3500220820000e01410024
:10417c00210320008e8040008001eb0020002000f5
:10418c008e010700e10f5000a0003a001e80900045
:10419c00e30f500099003400200320000e00400073
:1041ac0010409000e94f500083003a00200320009b
:1041bc000e004000204090000080fb00201798006b
:1041cc00200320000e004000304090000080fb00d7
:1041dc00101798002e109000c800dd001e109000e3
:1041ec0000804000301798003e109000cf80de0019
:1041fc003df10700201f9900311f99003e109000df
:10420c000000e00007003d000200200003782400bd
:10421c002e189100be189100a3f10700201f9900e1
:10422c00311f99002e189100be189100300f980084
:10423c00410f980002002000433b24003e089000f0
:10424c00ce089000f5f1070002002000035824006e
:10425c0050f10700300f9800410f98000200200029
:10426c00433b24003e089000ce0890001ff207004c
:10427c000000e00007003c006011b8003e08900010
:10428c00ce08900085f107000000e0000100350029
:10429c00030037000000eb006017980085ff370023
:1042ac000200200003f82b001e089000ae089000be
:1042bc007af107000000e000010032000400370032
:1042cc003e099000ce099000120f9800230f980021
:1042dc001e099000ae0990003e089000ce08900098
:1042ec0070f1070070079800010f98000200200081
:1042fc00433324007e0090008e089000fbf10700f1
:10430c000000e00001003c00070037000200200024
:10431c00433b24007e0090008e08900061f1070062
:10432c0070079800010f98000200200043332c0006
:10433c007e0090008e08900058f107000000e0000d
:10434c00010035000700370002002000433b240029
:10435c007e0090008e08900053f1070070079800c3
:10436c00010f98007e0190008e0990007e0890004d
:10437c008e1090004cf10700700f980001179800f8
:10438c0002002000433b24007e0890008e10900019
:10439c0000f10700500f9800610f98003e08900044
:1043ac00ce089000100f9800210f980010002000ec
:1043bc006017980013003700200320000e00400007
:1043cc0090409000a0c4b30080cf50000d003a0084
:1043dc00200320000e00400020409000e14f5000d0
:1043ec0003003a0010002000401798000500370029
:1043fc000000eb0040179800020037000000eb00b3
:10440c00601798000000eb00108798000013200044
:10441c000e0040003ff007000e1991009e1991000c
:10442c006e109100fe109100000051008180590027
:10443c00adf00700008fbe0002742c00e3a5240031
:10444c001e00be00d3f00700008fbe00004e80009f
:10445c00cf80de00a4f007001e01be000ff10700a4
:10446c000000e000030034006e009000e10f5000eb
:10447c0037003a00410d20008e8040006e119000f4
:10448c00821f78005e099000ee099000829fbe00aa
:10449c00c0e42900801f78000100780050f6070066
:1044ac00e8875700400d20000e0040000e01070069
:1044bc0040079800410d20008e804000ce019000f6
:1044cc00831f78006e109000801f78005e099000aa
:1044dc00ee099000829fbe00f0e52900801f780055
:1044ec00010078003ef60700ea8757000200200022
:1044fc0003f82b001e089000ae0890007df1070019
:10450c000000e00001003a00070037005e10900048
:10451c00e10f500004003200410d20008e8040005d
:10452c0010002000e3010700c01220000e00400024
:10453c00f8ef07006e009000e10f500002003a0007
:10454c000000eb00600798000000eb00601798007b
:10455c00410820008e8040000001eb00100020007c
:10456c003e0007000000e000190032004008200067
:10457c000e0040009040780060e729001040780061
:10458c0080cf500006003a0081e72900100020007f
:10459c00c801070010002000501798000c003700cd
:1045ac00400820000e0040009040780090e8290060
:1045bc001040780080cf500005003a00b1e8290087
:1045cc0010002000bb0107000000eb005017980002
:1045dc001e00be0011000700e10f500003003a005e
:1045ec0010002000c5040700020037001000200056
:1045fc00cf04070020002000da040700e10f500070
:10460c0003003a0020002000bc040700a9fe37007c
:10461c0020002000c6040700a6fe37000600fa00a2
:10462c0010079800210798001e009000ae00900023
:10463c0032f10700000f78001e00780022002000e5
:10464c00110009000200d8008000fd00000f780066
:10465c001e0078000080fa00000006000a00fa0034
:10466c00200798003107980042079800d0c0b3008b
:10467c00204798000000eb00c04d8800e300470085
:10468c002e009000340107000000e00048003200ca
:10469c004e009000e10f500009003a00be4090001f
:1046ac00100020004b0107003e409000ed4f5000e1
:1046bc0003003a00a1c0b300100020004501070020
:1046cc00be4090002e40900080cf50001f00320062
:1046dc003e409000e84f50000f0032003e409000ea
:1046ec00ea4f50000c003200d14d8000f004200045
:1046fc00808f500008003c00d14d80003e4190005e
:10470c008091200000804000024878000100e80001
:10471c00d04d880009003700d04d80000000e0002b
:10472c00060034003e409000e84f500003003a0071
:10473c00d04d80000000e900d04d8800be009000f4
:10474c000040eb0080487800190037001000200072
:10475c00c04d8800d14d80008091200080804000a9
:10476c000040eb00804878000000eb00000f780060
:10477c000a0037001e007800800078003e00900090
:10478c00008140009e007800809120000080400055
:10479c0010407800004978001e0fe800d04d8000d2
:1047ac009e0f1000f3ff34000000eb00d04d88008a
:1047bc00c04d80000080fa00000006000c00fa00da
:1047cc00200798003107980042079800530798007b
:1047dc0000cab300204798000000eb00e04d8800b1
:1047ec00e30047002e009000db0007000000e00013
:1047fc003a0032005e009000e10f500003003a00d6
:10480c00be40900010002000f2000700be40900057
:10481c002e40900080cf500012003200f14d8000ed
:10482c00f0042000808f500007003c00f14d800008
:10483c003e419000809620000080400002487800a5
:10484c000100e800f04d8800be0090000040eb0035
:10485c0080487800f14d80004e00900001087800ef
:10486c001e003700f14d80003e41900080962000e4
:10487c0000804000024878000100e800f04d8800fc
:10488c000000eb00000f78000a0037001e007800d3
:10489c00800078003e009000008140009e0078006f
:1048ac00809620000080400010407800004978007d
:1048bc001e0fe800f04d80009e0f1000f3ff350036
:1048cc00f14d80004e009000010878000000eb00d4
:1048dc00f04d880010002000e04d8800e04d800075
:1048ec000080fa00000006000a00fa003007980069
:1048fc000000eb00200798003e00900073f50700c5
:10490c00100798000000eb00000f78002c00370017
:10491c001e007800800078003e009000008040006f
:10492c0090407800a0c2b30080cf50002700320026
:10493c001e007800800078003e009000008040004f
:10494c00104078000080fb004007980040022000d7
:10495c00ce009000808f500018003200a002200082
:10496c00ce009000808f5000140032002e0090007a
:10497c000000e00008003a001e007800800078007b
:10498c003e00900000804000104078000080fb004a
:10499c0020079800090037001e007800800078007e
:1049ac003e00900000804000104078008080fb00aa
:1049bc002e00900001006800200798001e0fe800f0
:1049cc001e0090009e0f1000d1ff35002e009000ad
:1049dc000080fa00000006000200fa000000eb0064
:1049ec00000f7800270037009e0178001e00780029
:1049fc004700dd00800078004081200000804000ee
:104a0c0000017800c318dd004080200000804000c9
:104a1c00020878001e0078004300dd008080e8006a
:104a2c0040802000808040000000eb00800878006f
:104a3c001e0078004300dd00e400400040802000b0
:104a4c00808040000000eb00800878001e00780099
:104a5c004300dd00e60040004080200080804000e4
:104a6c00f0072000800878001e00780080004000cd
:104a7c0040912000808040000000eb00800878000e
:104a8c001e0fe800100020009e0f1000d6ff34000f
:104a9c00700120004011880021e2a80020a2a9008a
:104aac002062a90000402000101188008560a90038
:104abc008580a900910a200091407800f0c8b300cd
:104acc0000c0600001c6b30001407000a9e0b7004f
:104adc00a10a20009140780080cfb30000c0600094
:104aec000014a000aae0b7009560a8009580a9006a
:104afc0070012000c011880031e2a80030a2a9008a
:104b0c003062a900004020009011880087c0a900e5
:104b1c0087e0a900310b20009140780080cfb300d2
:104b2c0000c060006040b300b3e0b700310b200060
:104b3c0091407800f0c8b30000c0600001c2b3001f
:104b4c0001407000b3e0b70097c0a80097e0a9003f
:104b5c000080fa00000006000a00fa001007980016
:104b6c00210798001e009000400798004e0090000e
:104b7c00e10f5000090032004e009000e20f50008f
:104b8c0006003200ae0090000040eb008048780038
:104b9c000000eb00300798000b0037001e0090005f
:104bac004300dd0080007800408020006800500049
:104bbc00808040002e009000ed020700000f78006e
:104bcc001e007800300798003e0090000080fa002c
:104bdc00000006000c00fa001007980041479800ee
:104bec001e009000400798004e009000e10f50000e
:104bfc00040032004e009000e20f5000080032001a
:104c0c000e00370023c2bf000080fb000000d10063
:104c1c00614060000080fb00000f78000900370045
:104c2c0033c2bf000080fb000000d1006140600077
:104c3c000080fb00000f78000200370010002000fd
:104c4c00000f78001e00e00015003a001e009000d6
:104c5c00500798005e009000e10f500004003200f5
:104c6c005e009000e20f5000070032000c0037008d
:104c7c004e4090000080fb002011880010002000a6
:104c8c0030079800080037004e4090000080fb0071
:104c9c00a011880010002000300798000200370097
:104cac000000eb00300798003e0090000080fa00f6
:104cbc00000006000600fa00100798002107980073
:104ccc000000eb00000f78000b0037001e0078008e
:104cdc00800078002e00900000804000104078008a
:104cec00804078001e009000baff07000000e00032
:104cfc00010032001e0fe8001e00780080007800d2
:104d0c002e00900000804000104078000004e0006d
:104d1c00eeff3a000000eb000080fa0000000600f5
:104d2c000800fa00100798001e0090003007980049
:104d3c003e009000e10f5000060032003e00900053
:104d4c00e20f5000030032000000eb002007980037
:104d5c000a0037001e0090004300dd008000780040
:104d6c00408020006800500000804000ac0207002a
:104d7c00000f78001e007800200798002e0090008d
:104d8c000080fa00000006000600fa0010079800e8
:104d9c001e009000200798002e009000e10f50009c
:104dac00040032002e009000e20f50000800320088
:104dbc000e00370023c2bf000080fb000000d100b2
:104dcc00614060000080fb00000f78000900370094
:104ddc0033c2bf000080fb000000d10061406000c6
:104dec000080fb00000f780002003700100020004c
:104dfc00000f78001e0078000080fa00000006000a
:104e0c000600fa00000f78001e00780020079800ba
:104e1c002e009000e10f5000040032002e00900094
:104e2c00e20f5000080032000e0037001e00780020
:104e3c00800040004091200000804000100078006d
:104e4c0010079800090037001e0078008000400011
:104e5c00409120000080400010007800100798005e
:104e6c00020037000000eb00100798001e009000b5
:104e7c000080fa00000006000400fa00000f780021
:104e8c001e007800100798001e009000e10f5000e3
:104e9c00040032001e009000e20f500001003200ae
:104eac00060037001e007800800040004091200072
:104ebc00808040000000eb00800878000080fa0041
:104ecc00000006000800fa00100798001e00900071
:104edc00200798002e009000e10f500004003200d3
:104eec002e009000e20f5000010032001d00370030
:104efc001e0090004300dd00800078004080200000
:104f0c0068005000008040003b0207001e0090002b
:104f1c00300798003e009000e10f50000600320070
:104f2c003e009000e20f50000a0032000d003700e6
:104f3c0030118000000f780022c2bf006140600079
:104f4c000004e000faff3a0006003700b0118000c0
:104f5c00000f780032c2bf00614060000004e00026
:104f6c00faff3a000080fa00000006000400fa0084
:104f7c00000f78001e007800100798001e009000ab
:104f8c00e10f5000040032001e009000e20f5000b0
:104f9c0006003200090037002342a900000000007f
:104fac002342a80000000000040037003342a9008f
:104fbc00000000003342a800000000000080fa004e
:104fcc0000000600809fbe000000fa000040800038
:104fdc001140800061004000e080480000408800e3
:104fec00114088008580a9000080fa004f00be00a7
:104ffc0000400600809fbe000000fa00140037003d
:10500c00304080008000e8005040800080806000cc
:10501c0040408000808f500003003a0010002000b8
:10502c00a04888000a0037002140800030408000f2
:10503c008080400030118000804878003040800033
:10504c008000e80050408000008060003040880004
:10505c0022c2bf00614060000004e000e8ff3a009b
:10506c008560a9000080fa004f00be0000400600d9
:10507c00809fbe000000fa000040800011408000bc
:10508c0061004000e080480000408800114088002a
:10509c0087e0a9000080fa004f00be000040060027
:1050ac00809fbe000000fa001400370070408000a2
:1050bc008000e8009040800080806000804080008c
:1050cc00808f500003003a0010002000b048880088
:1050dc000a003700614080007040800080804000f2
:1050ec00b011800080487800704080008000e8009b
:1050fc0090408000008060007040880032c2bf0089
:10510c00614060000004e000e8ff3a0087c0a9009d
:0c511c000080fa004f00be0000400600ba
:020000040000fa
:10512800b80900000800000000000000180900008d
:10513800a0000000020000000000000000000000c5
:105148000000000000000000000000000000000057
:105158000000000000000000000000000000000047
:105168000000000000000000000000000000000037
:105178000000000000000000000000000000000027
:105188000000000000000000000000000000000017
:105198000000000000000000000000000000000007
:1051a80000000000000000000000000000000000f7
:1051b80000000000000000000000000000000000e7
:1051c80000000000000000000000000000000000d7
:1051d80000000000000000000000000000000000c7
:1051e80000000000000000000000000000000000b7
:1051f80000000000000000000000000000000000a7
:105208000000000000000000000000000000000096
:10521800000800001801000000000000c20900009a
:10522800d0010000020000000100000000000000a2
:10523800000008000000000000000000004000001e
:105248000000000000000000000200000000000054
:1052580000000000100000000000000000008000b6
:105268000000000000000000000004000000000032
:105278000000000000200000000000000000000006
:10528800000100000000000000000000080000000d
:1052980000000000000040000000000000000000c6
:1052a80000000200000000000000000000100000e4
:1052b8000000000000000000800000000000000066
:1052c80000000000040000000000000000002000b2
:1052d80000000000000000000000010000000000c5
:1052e80000000000000800000000000000000000ae
:1052f8004000000000000000000000000200000064
:105308000000000000001000000000000000000085
:1053180000800100000000000000000000100000f4
:105328000000000000000000000100000000000074
:105338000000000010000000000000000000000055
:105348000100000000000000000010000000000044
:105358000000000000000100000000000000000044
:105368000010000000000000000000000001000024
:105378000000000000000000100000000000000015
:105388000000000001000000000000000000100004
:105398000000000000000000000001000000000004
:1053a80000000000001000000000000000000000e5
:1053b80000010000000000000000000010010000d3
:1053c80000000000000000000a00000000000000cb
:1053d80000006400000000000000000000e8030076
:1053e800000000000000000010270000000000007e
:1053f8000000a000860100000000000000404200fc
:105408000f000000000000008096980000000000d7
:1054180000000000e1f50500000000000000ca00df
:105428009a3b00000000000000e40b00540200005a
:1054380000000000e8764800170000000000100097
:10544800a5d4e8000000000000a072004e18090072
:1054580000000000407a1000f35a000000008000ad
:10546800c6a47e008d0300000000c1006ff2860014
:1054780023000000008a5d007845630001000000f9
:1054880064a7b300b6e00d000000e800890423001b
:10549800c78a0000f20c00002a0000000200000089
:1054a800286e75006c6c29000030310032333400ee
:1054b800353637003839410042434400454600003c
:1054c8003031320033343500363738003961620004
:1054d8006364650066000000920b00006001000034
:1054e800020000000000000000000000f03f000083
:1054f8000000a0009999b9003f0000000040e100b9
:105508007a843f0000000000e04d6200503f000038
:105518000000e000e2361a003f0000000080b500fd
:10552800f8e43e0000000000a0f7c600b03e00000e
:105538000000a000f2d77a003e00000000e08e00d4
:1055480079453e0000000000e00b2e00113e0000ef
:105558000000e000df7cdb003d0000000000a1004f
:105568009cc73b0000000000004c4800b439000014
:1055780000000000206ca1003700000000000000bf
:105588000000000000000000000000000000000013
:105598000000000000000000000000000000000003
:1055a80000000000000000000000000000000000f3
:1055b80000000000000000000000000000000000e3
:1055c80000000000000000000000000000000000d3
:1055d800000000000000f0003f0000000000000094
:1055e80000244000000000000000000059400000b6
:1055f8000000000000408f00400000000000000094
:1056080088c340000000000000006a00f840000065
:105618000000000080842e00410000000000d0003f
:1056280012634100000000000084d7009741000089
:105638000000000065cdcd004100000000205f00a3
:10564800a002420000000000801daf0015440000c9
:1056580000004000593e29004600000000000000fc
:1056680000f07f000000000000000000f07f000054
:10567800000000000000f0007f00000000000000b3
:1056880000f07f000000000000000000f07f000034
:10569800000000000000f0007f0000000000000093
:1056a80000f07f000000000000000000f07f000014
:1056b800000000000000f0007f0000001c0d00004a
:1056c80002000000000000001e0d000002000000a3
:1056d80000000000200d0000020000000000000093
:1056e800220d00000200000002000000010000007e
:1056f800240d00000200000000000000000000006f
:020000040000fa
:105708000600fa00004f7800110798001e0090006c
:10571800440007000000e000030032000000eb0036
:1057280020079800100037001e00900090007800b5
:105738001e00900010009000008040001e48780075
:105748001e009000100090008000e8001e009000ed
:1057580030009000808060001e00900011009800ca
:1057680010002000200798002e0090000080fa000a
:10577800000006000600fa00000f780011079800e4
:105788001e0090003b0007000000e0000600320009
:105798009e0078000040eb00804878000000eb0095
:1057a80020079800120037001e0090009000780033
:1057b8001e0090002000900000804000904078007b
:1057c8001e007800014878001e009000200090001c
:1057d8008000e8001e00900030009000808060008b
:1057e8001e0090002100980010002000200798005b
:1057f8002e0090000080fa00000006000200fa0067
:10580800000f78009e0078000000eb00a0009800d0
:105818009e0078000000eb00900098000080fa00dd
:10582800000006000400fa00000f78001e0078004f
:10583800100090008000e8001e0078003000900002
:10584800808060001e00780020009000808f50004b
:1058580003003a00100020001007980002003700eb
:105868000000eb00100798001e0090000080fa006e
:10587800000006000400fa00000f78001e007800ff
:10588800a00090001e00780010009000808f50004b
:1058980003003a00100020001007980002003700ab
:1058a8000000eb00100798001e0090000080fa002e
:1058b800000006000200fa00000f78001e007800c1
:1058c800900090001e00780020009000808050001a
:1058d8001e00780030009000008060000080fa0010
:1058e800000006000000fa00c902a900c922a900a8
:1058f800c8c2a800c8e2a8000080fa00000006009c
:105908000200fa00000f7800100020009e0f10001f
:1059180002003a00cd02a900040037002000200050
:105928009e0f100001003a00cd22a9000080fa0065
:10593800000006000200fa00000f780010002000a6
:105948009e0f100002003a00cd02a80004003700a4
:10595800200020009e0f100001003a00cd22a80070
:105968000080fa00000006000600fa0020079800f0
:105978000000eb00100798000000eb00000f780013
:105988002e009000e10f500007003a00cac2bf0085
:105998000080fb004600de00614060000080fb00e4
:1059a800000f7800080037002e009000e20f50002a
:1059b80005003a00cac2bf000080fb004700de00b5
:1059c8000080fb00000f7800100020009e0f1000e0
:1059d80002003a000000eb00100798001e00e000eb
:1059e80002003a0010002000100798001e009000e6
:0859f8000080fa000000060027
:020000040000fa
:045a00000000fe00a4
:00000001FF
